:020000000528D1
:1000080092298B138312031383120313850186012C
:100018008316FF30831603138500FF308600831292
:100028008B138730831681008312C3308312031326
:10003800CA00CB018100A0308B00CC01FF30CF017A
:10004800D001D100D2002A2983120313CE00031055
:100058004C0D4F3E840083134D088000840A4E08DF
:100068008000CC0A4C08013A0319CC0103104C0D4E
:1000780083134F3E84000008840A000403193528BE
:10008800801B352800088A00840300088200831238
:1000980003133E083F04031D5228592801308312D8
:1000A8000313BE02031CBF034B280800831203136B
:1000B80037083804031D61287D280A30831203138A
:1000C800B9003908003A031D6A28762883120313F9
:1000D800CE01FA30CD000000CD0B6F2800000130B2
:1000E800B9026528013083120313B702031CB80351
:1000F8005A28080083120313851508008312031376
:10010800851108008312031305153E0EF039860485
:100118000F3886050511080082208312031337085B
:10012800BE00BE0E0F30BE058620831203133708AB
:10013800BE00862083120313BF013230BE004B205D
:1001480008007E20831203132B08BE00BE0E0F305A
:10015800BE058620831203132B08BE008620831257
:100168000313BF013230BE004B200800831603136F
:1001780006128612061386138511051183120313BE
:10018800B8010A30B7005A208220033083120313C3
:10019800BE00862083120313B8010530B7005A2029
:1001A800033083120313BE00862083120313BF019A
:1001B8006430BE004B20033083120313BE00862038
:1001C80083120313B8010530B7005A200230831296
:1001D8000313BE00862083120313BF013230BE0012
:1001E8004B20283083120313B70090200830831265
:1001F8000313B70090200F3083120313B700902029
:10020800013083120313B7009020063083120313C2
:10021800B7009020831203132C088A002B08820051
:10022800831203132E080139B700B70EB70DB70DA7
:10023800C030B7058030B7042D083F39B704902087
:10024800831203132C088A002B08820007308312BC
:1002580003139F000130AC003630AB0000308A0039
:10026800BA30820083120313A201A301A40103116F
:1002780003193F2940298C2983120313A20A031466
:10028800A21B482922080F3C031C4B295A29831218
:100298000313A201A30A0314A31B54292308013C36
:1002A800031C57295A2983120313A3012208AD00FE
:1002B8002308AE000130AC006630AB0001308A0084
:1002C80014308200831203132408AB00A520831284
:1002D8000313A40AA501A6010310A61B7B2900305D
:1002E8002602031C7B29031D7B2964302502031C7D
:1002F8007E298B2983120313CE01FA30CD0000002A
:10030800CD0B83290000A50A0319A60A70293B29E9
:100318008312031321088A0020088200FF00030EBD
:100328008312031383120313C400C40E0A08C50002
:100338000408C6000B1DB1294A0881005030CB07BC
:10034800B4300318013EFF3A013ECA000B11FF30DA
:10035800D21BB129D107031CD2077C08C7007D082E
:10036800C8007E08C9004908FE004808FD00470883
:10037800FC004608840045088A0044088300FF0EF4
:040388007F0E0900DB
:02400E00103F61
:00000001FF
